:100000000C945C000C94F6030C9423040C94840070
:100010000C9484000C9484000C9484000C94840050
:100020000C9484000C9484000C9484000C94840040
:100030000C9484000C9484000C9484000C94840030
:100040000C9450040C9484000C9449050C94840086
:100050000C9484000C9484000C9484000C94840010
:100060000C9484000C948400000024272A000025AE
:10007000282B000023262904040404040404040299
:100080000202020202030303030303010204081035
:100090002040800102040810200102040810200002
:1000A0000000070002010000030406000000000039
:1000B000000000005802E90211241FBECFEFD4E077
:1000C000DEBFCDBF11E0A0E0B1E0E8E2FEE002C09B
:1000D00005900D92A830B107D9F712E0A8E0B1E081
:1000E00001C01D92A031B107E1F710E0C8EBD0E0EC
:1000F00004C02297FE010E940E07C43BD107C9F736
:100100000E94E2020C9412070C940000FC01448748
:100110005587668777870895CF93DF93EC01EC8D41
:10012000FD8D9081888D809589238083E8A1F9A138
:1001300090818E8D809589238083ECA1FDA1908193
:100140008E8D809589238083E8A1F9A180819E8D81
:10015000892B8083E8A1F9A190818E8D80958923D8
:100160008083EC8DFD8D8081988D892B8083EAA121
:10017000FBA180816E8D90E0262F30E082239323B7
:10018000892BB1F42C893D894E895F8988859985B1
:10019000AA85BB85281739074A075B0748F42F5FF4
:1001A0003F4F4F4F5F4F2C8B3D8B4E8B5F8BDFCF85
:1001B0002C893D894E895F8988859985AA85BB856B
:1001C00082179307A407B50708F440C0ECA1FDA16E
:1001D0008081682B6083E8A1F9A180819E8D892BA5
:1001E0008083E8A1F9A190818E8D809589238083F9
:1001F000ECA1FDA190818E8D809589238083EC8D6B
:10020000FD8D9081888D809589238083EAA1FBA153
:10021000208130E08E8D90E028233923232BE1F0DC
:100220002C893D894E895F8988859985AA85BB85FA
:10023000281739074A075B0778F42F5F3F4F4F4F66
:100240005F4F2C8B3D8B4E8B5F8BE0CF2EEF3FEFC4
:10025000C901DF91CF9108952C893D894E895F892D
:1002600088859985AA85BB85281739074A075B07C2
:1002700068F721E030E0ECCFEF92FF920F931F93ED
:10028000CF93DF93EC01062F1C8A1D8A1E8A1F8ADA
:10029000662329F420E030E040E050E07FC0888110
:1002A000998197FF05C02FEF3FEF4FEF5FEF76C0CB
:1002B00010E0CE010E948C0097FF05C02EEF3FEFAB
:1002C0004FEF5FEF6BC01F5F101798F30E94C004E1
:1002D000288939894A895B89621B730B840B950BCA
:1002E0002C853D854E855F852617370748075907BA
:1002F000C0F52C893D894E895F896A817B818C811B
:100300009D81261737074807590721F4EE24FF245B
:10031000870106C079018A01E61AF70A080B190B52
:100320000E94B7052DEC3CEC4CEC5DE30E944506C9
:100330000E948605882777FD8095982FE616F70698
:100340000807190770F48FEF9FEFAFEFBFE08A83C4
:100350009B83AC83BD830E94C004688B798B8A8B9E
:100360009B8B2C893D894E895F898A819B81AC81D9
:10037000BD81281739074A075B0720F42A833B838E
:100380004C835D832C893D894E895F898A819B815D
:10039000AC81BD81281B390B4A0B5B0BB901CA012B
:1003A000DF91CF911F910F91FF90EF900895CF9320
:1003B000DF93EC0181E090E09983888386E391E00C
:1003C0009F838E8380EF9AEBA4E0B0E088879987C3
:1003D000AA87BB8780E29EE4A0E0B0E08C879D877F
:1003E000AE87BF87862F90E0FC01E557FF4FE49171
:1003F000E88F89589F4FFC016491698FE62FF0E0E8
:10040000E359FF4FE491EC8F1D8E842F90E0FC01A7
:10041000E557FF4FE491EE8F89589F4FFC014491BF
:100420004F8FE42FF0E0E359FF4FE491ECA31DA2BE
:10043000662321F48FEF9FEF99838883E98DF0E0A5
:10044000E859FF4FE491EA8F1B8E8F8D882321F4AA
:100450008FEF9FEF99838883EF8D8E2F90E0FC01C3
:10046000E859FF4FE491E8A319A2FC01E359FF4FBB
:10047000E491ECA31DA28E589F4FFC0184918AA3A6
:100480001BA2EA8DFB8D8081988D892B80838FEF55
:100490009FEFAFEFBFE08A839B83AC83BD830E9455
:1004A000C004688B798B8A8B9B8BDF91CF910895E9
:1004B00042E064E088E091E00E94D70145E064E01A
:1004C0008EE291E00E94D70148E064E084E591E08B
:1004D0000E94D70108952F923F924F925F926F92A0
:1004E0007F928F929F92AF92BF92CF92DF92EF92C4
:1004F000FF920F931F930E94C0047B018C016EE159
:1005000088E091E00E943C015B016C016EE18EE2AB
:1005100091E00E943C013B014C016EE184E591E0D9
:100520000E943C011B012C010E94C004AB01BC01D4
:100530004E195F09600B710B0AE711E0C8010E94B8
:10054000C00380E0E82E81E0F82EB701C8010E94C8
:10055000F902B601A501C8010E94C403B701C80190
:100560000E94F902B401A301C8010E94C403B701AB
:10057000C8010E94F902B201A101C8010E94EB0367
:100580001F910F91FF90EF90DF90CF90BF90AF90B1
:100590009F908F907F906F905F904F903F902F90A3
:1005A00008954FEF5FEF6FEF7FEF88E091E00E94DB
:1005B000860040E05BE460E070E08AE791E00E9442
:1005C000F40208950E94CE040E94D1020E946B02A0
:1005D000FDCF86E091E090937B0180937A010895AE
:1005E000862F0E9441050895CB01BA010E9408059B
:1005F00008950F931F93CF93DF938C01EB0109C0F4
:100600002196D801ED91FC910190F081E02DC80177
:10061000099568816623A1F7DF91CF911F910F9112
:1006200008950F931F938C01DC01ED91FC910190D3
:10063000F081E02D6DE00995D801ED91FC910190DC
:10064000F081E02D6AE0C80109951F910F9108958E
:100650002F923F924F925F926F927F928F929F92D2
:10066000AF92BF92CF92DF92EF92FF920F931F93C0
:10067000DF93CF93CDB7DEB7A0970FB6F894DEBF68
:100680000FBECDBF1C016A017B01411551056105FB
:10069000710549F4DC01ED91FC910190F081E02DB0
:1006A00060E3099554C0882499245401422E5524AE
:1006B0006624772401E010E00C0F1D1F080D191DA2
:1006C000C701B601A30192010E94BB06F801608335
:1006D0000894811C911CA11CB11CC701B601A30187
:1006E00092010E94BB06C901DA016C017D01C114AF
:1006F000D104E104F104F1F681E0E82EF12CEC0ED6
:10070000FD1EE80CF91C3E010894611C711CD5010A
:10071000C4010197A109B1096C01C818D90814C016
:10072000F601EE0DFF1D60816A3010F4605D01C0BE
:10073000695CD101ED91FC910190F081E02DC10146
:1007400009950894E108F1086E147F0449F7A09612
:100750000FB6F894DEBF0FBECDBFCF91DF911F91D2
:100760000F91FF90EF90DF90CF90BF90AF909F9050
:100770008F907F906F905F904F903F902F90089553
:100780002AE00E9428030895EF92FF920F931F938F
:10079000CF93DF93EC017A018B0177FF0FC0E881E3
:1007A000F9810190F081E02D6DE209951095009599
:1007B000F094E094E11CF11C011D111D2AE0B80128
:1007C000A701CE010E942803DF91CF911F910F91C5
:1007D000FF90EF9008950F931F938C010E94C40324
:1007E000C8010E9411031F910F9108951F920F924B
:1007F0000FB60F9211242F933F934F935F936F93F4
:100800007F938F939F93AF93BF93EF93FF938091C9
:100810007C0190917D01892B29F0E0917C01F09180
:100820007D010995FF91EF91BF91AF919F918F91BC
:100830007F916F915F914F913F912F910F900FBEDC
:100840000F901F9018951F920F920FB60F921124C0
:100850002F933F934F935F936F937F938F939F93C8
:10086000AF93BF93EF93FF9380917E0190917F01AF
:10087000892B29F0E0917E01F0917F010995FF918C
:10088000EF91BF91AF919F918F917F916F915F9108
:100890004F913F912F910F900FBE0F901F90189581
:1008A0001F920F920FB60F9211242F938F939F9345
:1008B000AF93BF938091800190918101A0918201BB
:1008C000B09183010196A11DB11D80938001909389
:1008D0008101A0938201B093830180918401909162
:1008E0008501A0918601B09187018050904CAF4F57
:1008F000BF4F8093840190938501A0938601B093AC
:10090000870127C08091840190918501A091860183
:10091000B091870180549F41A040B04080938401F2
:1009200090938501A0938601B093870180918801FF
:1009300090918901A0918A01B0918B010196A11D2E
:10094000B11D8093880190938901A0938A01B0938F
:100950008B018091840190918501A0918601B091D5
:10096000870181549F41A040B04060F6BF91AF9194
:100970009F918F912F910F900FBE0F901F90189500
:100980008FB7F894209188013091890140918A01B4
:1009900050918B018FBFB901CA010895789484B535
:1009A000826084BD84B5816084BD85B5826085BD6B
:1009B00085B5816085BDEEE6F0E080818160808351
:1009C000E1E8F0E0808182608083808181608083C3
:1009D000E0E8F0E0808181608083E1EBF0E08081FD
:1009E00084608083E0EBF0E0808181608083EAE7CF
:1009F000F0E0808184608083808182608083808158
:100A0000816080838081806880831092C100089516
:100A1000EF92FF920F931F937B018C0122E030E055
:100A200040E050E00E94DD06205E3E45484F5F4FAB
:100A3000CA01B901A80197010E94DD06C901DA01C6
:100A40000197A109B109292F3A2F4B2F552747FDAF
:100A50005A950196A11DB11D2093C5008150809328
:100A6000C400E1ECF0E08081806180838081886057
:100A700080838081806880831F910F91FF90EF9029
:100A80000895982F8091C00085FFFCCF9093C600F9
:100A900008951F920F920FB60F9211242F933F9338
:100AA0004F935F936F937F938F939F93AF93BF9376
:100AB000EF93FF934091C600E0918C01F0918D017E
:100AC000CF01019660E870E00E94A8069C01809129
:100AD0008E0190918F012817390739F0E057FE4FAA
:100AE000408330938D0120938C01FF91EF91BF9152
:100AF000AF919F918F917F916F915F914F913F91B6
:100B00002F910F900FBE0F901F90189504D06894EE
:100B1000B111B5C0089598D088F09F5790F0B92FC3
:100B20009927B751A0F0D1F0660F771F881F991F42
:100B30001AF0BA95C9F712C0B13081F09FD0B1E078
:100B400008959CC0672F782F8827B85F39F0B93F88
:100B5000CCF3869577956795B395D9F73EF4909544
:100B60008095709561957F4F8F4F9F4F0895E894C2
:100B700009C097FB3EF490958095709561957F4FE5
:100B80008F4F9F4F9923A9F0F92F96E9BB27939593
:100B9000F695879577956795B795F111F8CFFAF4A3
:100BA000BB0F11F460FF1BC06F5F7F4F8F4F9F4FD4
:100BB00016C0882311F096E911C0772321F09EE832
:100BC000872F762F05C0662371F096E8862F70E098
:100BD00060E02AF09A95660F771F881FDAF7880F72
:100BE0009695879597F9089597F99F6780E870E043
:100BF00060E008959FEF80EC089500240A94161693
:100C0000170618060906089500240A9412161306FA
:100C1000140605060895092E0394000C11F4882388
:100C200052F0BB0F40F4BF2B11F460FF04C06F5FA4
:100C30007F4F8F4F9F4F089557FD9058440F551F7A
:100C400059F05F3F71F04795880F97FB991F61F04E
:100C50009F3F79F087950895121613061406551FC5
:100C6000F2CF4695F1DF08C0161617061806991F31
:100C7000F1CF86957105610508940895E894BB2726
:100C800066277727CB0197F908950BD0C4CFB5DF3E
:100C900028F0BADF18F0952309F0A6CFABCF1124C6
:100CA000EECFCADFA0F3959FD1F3950F50E0551F0B
:100CB000629FF001729FBB27F00DB11D639FAA27B1
:100CC000F00DB11DAA1F649F6627B00DA11D661F00
:100CD000829F2227B00DA11D621F739FB00DA11D21
:100CE000621F839FA00D611D221F749F3327A00DDB
:100CF000611D231F849F600D211D822F762F6A2F77
:100D000011249F5750408AF0E1F088234AF0EE0FFB
:100D1000FF1FBB1F661F771F881F91505040A9F708
:100D20009E3F510570F060CFAACF5F3FECF3983E35
:100D3000DCF3869577956795B795F795E7959F5F6F
:100D4000C1F7FE2B880F911D9695879597F9089509
:100D500097FB092E07260AD077FD04D049D006D08C
:100D600000201AF4709561957F4F0895F6F79095DD
:100D700081959F4F0895A1E21A2EAA1BBB1BFD016E
:100D80000DC0AA1FBB1FEE1FFF1FA217B307E4076A
:100D9000F50720F0A21BB30BE40BF50B661F771FC2
:100DA000881F991F1A9469F76095709580959095A2
:100DB0009B01AC01BD01CF01089597FB092E0526CB
:100DC0000ED057FD04D0D7DF0AD0001C38F4509560
:100DD0004095309521953F4F4F4F5F4F0895F6F75F
:100DE00090958095709561957F4F8F4F9F4F089597
:100DF000AA1BBB1B51E107C0AA1FBB1FA617B70741
:100E000010F0A61BB70B881F991F5A95A9F780955C
:100E10009095BC01CD010895EE0FFF1F0590F49150
:080E2000E02D0994F894FFCFC6
:080E2800090000000000F002C7
:00000001FF
